:030000000200CE2D
:1000CE0075810875F67875847875858712003512F6
:1000DE0000B7D2AFE58953891F438910C2AFE590AF
:1000EE00A28013F4F521A281B39200C20154F092C2
:1000FE00E17002D201D2AFC282D290A4A4A4A4A471
:10010E00A4A4A4A4A4D282C2997599003099FDC268
:10011E00AFE521700530000DC200D2AF1521C29996
:10012E0075990080E7D2AF7922D2ACDA02B2822082
:10013E00ACFD30010C7B103099FDC299759900DB36
:10014E00F63099FDA4A4A4C290758B00758DFFD2D4
:0A015E008E308FFDC28EC28F8082AA
:10002300C2AF5398FCD29B879909B92A02C2ACD2BA
:0B003300AF3275988875870079222293
:10005B00C2AFC2C4E5C5DC14308704F5228002F5BB
:10006B0026D2C0C2C17C02D2C3D2AF32DC143087DD
:10007B0004F5238002F527D2C1C2C07C03D2C3D2C0
:10008B00AF32DC14308704F5248002F528D2C0D2BD
:10009B00C17C04D2C3D2AF32308704F5258002F580
:1000AB0029C2C1C2C07C01D2C3D2AF3275C0807C21
:0F00BB00097822E4F608DCFC7C01D2C3D2EC22E7
:00000001FF
